:100000000C94BB070C94D8070C94D8070C94D80711
:100010000C94B0250C94D8070C94D8070C94D807EE
:100020000C94D8070C94D8070C94C42C0C94962DDF
:100030000C9410280C94D8070C94D8070C94D8076B
:100040000C94D8070C94D8070C94D8070C94D807B4
:100050000C94D8070C9489280C94D8070C94D807D2
:100060000C94D8070C94D8070C94D8070C94D80794
:100070000C94D8070C94D8070C94D8070C94D80784
:100080000C94D8070C94D8070C94D8070C94D80774
:100090000C94D8070C94D8070C94D8070C94D80764
:1000A0000C94D8070C94D8070C94D807470C470C2D
:1000B000730C730CDB0C060E060E060EF90C920D7B
:1000C000A30DA30D032E2A2E222F2A2E222F762EA9
:1000D000992E222FF02EFF2E20002D2D2D2D2D00BC
:1000E0002D5343524C0020002D2D2D2D2D002D433E
:1000F0004150530020002D2D2D2D2D002D4E554DFE
:100100004C002000556E646566696E65640020468B
:1001100050532020202000204D4F4241202020001D
:10012000204D454449412020002051574552545903
:10013000200020002D00414C54002D0057494E0056
:100140002D00435452002D00534846002D0020003E
:1001500000C0201008040201010101010101010396
:10016000070F1F3F7FFFFFFFFFFFFFFFFFFFFFFFA7
:10017000FFFFFF81819999999999991919FFFF01B9
:1001800001FFFFFFFFFFFFFFFFFFFF19199999997B
:100190009999990101FFFF81817F7FFFFF7F7F8117
:1001A00081FFFF9999999999999999F9F9FFFFFF19
:1001B000FFFFFFFFFFFFFFFFFFFFFF7F3F1F0F0757
:1001C0000301010101010101010204081020C00026
:1001D00000FF000000000000000000000000000020
:1001E0000000000000000103070F0F0F0F0F0F0F9B
:1001F0000F0F0F090909090909090908080F0F0854
:100200000809090909090909090F0F08080F0F0F43
:100210000F0F0F08080F0F0F0F0E0E09090E0E0F0C
:100220000F0F0F090909090909090909090F0F0F1A
:100230000F0F0F0F0F0F0F0703010000000000004A
:100240000000000000000000000000000000FF00AF
:1002500000FF00000000000000000000000000009F
:10026000000000000000000000000000000000008E
:10027000000000000000000000000000000000007E
:1002800000000000000000008040402020101010FE
:1002900010102020404080000000000000000000FE
:1002A000000000000000000000000000000000004E
:1002B000000000000000000000000000000000003E
:1002C0000000000000000000000000000000FF002F
:1002D00000FF00000000000000000000000000001F
:1002E000000000000000000000000000000000000E
:1002F00000000000000000000000000000000000FE
:10030000000000000000FE0100E02020E0000000EE
:100310000000E02020E00001FE00000000000000DE
:1003200000000000000000000000000000000000CD
:1003300000000000000000000000000000000000BD
:100340000000000000000000000000000000FF00AE
:1003500000FF00000000000000000000000000009E
:10036000000000000000000000000000000000008D
:10037000000000000000000000000000000000007D
:10038000E020202020203F0000F90101F90000F8C2
:100390000000F90101F900003F2020202020E000AA
:1003A000000000000000000000000000000000004D
:1003B000000000000000000000000000000000003D
:1003C0000000000000000000000000000000FF002E
:1003D00000FF00000000000000000000000000001E
:1003E000000000000000000000000000000000000D
:1003F00000000000000000000000000000000000FD
:10040000FF0000FC0000FF0101F110101F00003F81
:1004100000001F1010F30202F212121E0000FF0073
:1004200000000000000000000000000000000000CC
:1004300000000000000000000000000000000000BC
:100440000000000000000000000000000000FF00AD
:1004500000FF00000000000000000000000000009D
:10046000000000000000000000000000000000008C
:10047000000000000000000000000000000000007C
:100480000F00000F08080F00000909090909090FEA
:1004900000000F01010908080909090F00000F00F9
:1004A000000000000000000000000000000000004C
:1004B000000000000000000000000000000000003C
:1004C0000000000000000000000000000000FF002D
:1004D0000003040810204080808080808080C0E07D
:1004E000F0F8F8F8F8F8F8F8F8F8F8F8F8F8F8F894
:1004F000F8F8F8F8F8F8F8F8F8F8F8F8F8F8F8F87C
:10050000F8F8F8F8F8F8F8F8F8F8F8F8F8F8F8F86B
:10051000F8F8F8F8F8F8F8F8F8F8F8F8F8F8F8F85B
:10052000F8F8F8F8F8F8F8F8F8F8F8F8F8F8F8F84B
:10053000F8F8F8F8F8F8F8F8F8F8F8F8F8F8F8F043
:10054000E0C080808080808080402010080403000C
:100550000029001E001F002000210022002E002B79
:100560000014001A00080015001700005739000495
:10057000001600070009000A000000E1001D001B32
:1005800000060019000500B200E000E300E2004CA4
:10059000002A412C0028002D0023002400250026DD
:1005A0000027002A0001571C0018000C001200133D
:1005B00000310000000B000D000E000F00330002A0
:1005C00057460011001000360037003800E50028BB
:1005D000002C0003575000510052004F0029003AF0
:1005E000003B003C003D003E003F003900630057E7
:1005F00000560055005400AF002B005E005F006005
:1006000000610062000000E10059005A005B005CDC
:10061000005D00A800E000E300E2002A000100AA5B
:1006200000A9004000410042004300440045002A68
:1006300000AD000100010001000100A500005C0008
:10064000004700095CDF5C010001000100AE0053BF
:1006500000125C0100010001000100AC00AB0012BF
:10066000504A004E004B004D0029001E001F002084
:10067000002100220023002B0014001A000800159E
:100680000017002400E00004001600070009000A1B
:10069000000000E1001D001B000600190005002CF1
:1006A0000000000000000000002C002C002C0000C6
:1006B000000000000000000000000000000000003A
:1006C000000000000000000000000000000000002A
:1006D000000000000000000000000000000000001A
:1006E00000000000000000000000001350000000A7
:1006F00000E2002B0029001E001F00200021002224
:100700000023002B0004001A000800150017000B3E
:1007100000E1001D001600070009000A000000E0CB
:100720000000001B0006001900050010000000007A
:1007300000000000002C002C00140000000000004D
:1007400000000000000000000000000000000000A9
:100750000000000000000000000000000000000099
:100760000000000000000000000000000000000089
:1007700000000000000000105000000000E2002B0C
:1007800000B62020206162636465666768696A6BF1
:100790006C6D6E6F707172737475767778797A316B
:1007A0003233343536373839301413111D162D3D98
:1007B0005B5D5C233B27602C2E2FBC959697989908
:1007C0009A9B9C9D9E9FB5BFBE2020B9B710BAB81A
:1007D0001A1B1918BD2F2A2D2B20313233343536F0
:1007E000373839302E20BB20202020202020202008
:1007F00020202020202020202020202020202020F9
:1008000020202020202020202020202020202020E8
:1008100020202020202020202020202020202020D8
:10082000202020202020202020D6D7D8D9DADBDCB9
:10083000DD2020D520202020202020202020202046
:1008400020202020202020202020202020202020A8
:100850002020202020202020202020202020202098
:1008600020435341572053202020202020202020A7
:100870002020202020202020202020202020202078
:10088000C4C5C5C9CACACACACACACACACACACACAD9
:10089000CACBC5C5C600C1C7C7C7C7C7C7C7C7C7B3
:1008A000C7C7C7C7C7C7C7C7C7C7C200C000C1C778
:1008B000C7C7C7C7C7C7C7C3C7C7C7C7C7C7C7C7CC
:1008C000C7C7C200D400C8FF0080818283848586A8
:1008D0008788898A8B8C8D8E8F9091929394A0A11A
:1008E000A2A3A4A5A6A7A8A9AAABACADAEAFB0B170
:1008F000B2B3B4C00000AE00AF00DA1281FFD9F18C
:10090000DB20A4A62EAF00A0C000A1C800AED580F9
:10091000A83FD300408D1420000000000000003EDE
:100920005B4F5B3E003E6B4F6B3E001C3E7C3E1CB3
:1009300000183C7E3C18001C577D571C001C5E7F35
:100940005E1C0000183C180000FFE7C3E7FF000032
:100950001824180000FFE7DBE7FF0030483A060ED6
:1009600000262979292600407F05050700407F05DC
:10097000253F005A3CE73C5A007F3E1C1C080008FB
:100980001C1C3E7F0014227F2214005F5F005F5F0B
:100990000006097F017F00006689956A006040407B
:1009A00040600094A2FFA2940008047E0408001096
:1009B000207E20100008082A1C0800081C2A0808AD
:1009C000001E10101010000C1E0C1E0C0030383EC3
:1009D000383000060E3E0E06000000000000000049
:1009E000005F000000000700070000147F147F1460
:1009F00000242A7F2A120023130864620036495615
:100A0000205000000807030000001C2241000000E5
:100A100041221C00002A1C7F1C2A0008083E0808EE
:100A2000000080703000000808080808000000601E
:100A30006000002010080402003E5149453E0000BD
:100A4000427F4000007249494946002141494D33E7
:100A5000001814127F10002745454539003C4A49CB
:100A600049310041211109070036494949360046FC
:100A70004949291E00000014000000004034000015
:100A80000000081422410014141414140000412220
:100A90001408000201590906003E415D594E007CD0
:100AA0001211127C007F49494936003E41414122E2
:100AB000007F4141413E007F49494941007F09098A
:100AC0000901003E41415173007F0808087F000082
:100AD000417F4100002040413F01007F0814224136
:100AE000007F40404040007F021C027F007F0408DE
:100AF000107F003E4141413E007F09090906003E4A
:100B00004151215E007F0919294600264949493291
:100B10000003017F0103003F4040403F001F204091
:100B2000201F003F4038403F006314081463000357
:100B300004780403006159494D4300007F4141415D
:100B400000020408102000004141417F000402011E
:100B5000020400404040404000000307080000201D
:100B600054547840007F2844443800384444442892
:100B700000384444287F0038545454180000087E3C
:100B800009020018A4A49478007F080404780000E7
:100B9000447D4000002040403D00007F102844007C
:100BA0000000417F4000007C04780478007C080449
:100BB000047800384444443800FC182424180018F1
:100BC000242418FC007C08040408004854545424CD
:100BD0000004043F4424003C4040207C001C204092
:100BE000201C003C4030403C004428102844004C6D
:100BF0009090907C004464544C44000008364100BE
:100C000000000077000000004136080000020102E9
:100C10000402005C5653565C00C020100804020118
:100C20000101010101010103070F1F3F7FFFFFFFCA
:100C3000FFFFFFFFFF0101FFFF0101FFFF0101FFB8
:100C4000FF19199999999999990101FFFF81819942
:100C500099999999991919FFFFF9F9F9F90101F988
:100C6000F9F9F9FFFF9999999999999999F9F9FFE2
:100C7000FF19199999999999996767FFFFFFFFFFE4
:100C8000FFFFFF7F3F1F0F0703010101010101016A
:100C9000010204081020C01F0500021F001F0500EC
:100CA0001D17001F0500151F001F0500071C001F52
:100CB0000500171D001F05001F1D001F0500011F57
:100CC000001F05001F1F001F0500071F001F050054
:100CD0007077001F0500007700FF00000000000093
:100CE0000000000000000000000000000000010300
:100CF000070F0F0F0F08080F0F0E0E0F0F08080F2A
:100D00000F08080F0F0F0F0F0F08080F0F09090921
:100D100009F9F9090908080F0F0F0F0F0F08080F3D
:100D20000F0F0F0F0F090909090909090909090F0F
:100D30000F08080F0F0F0F0F0F08080F0F0F0F07E7
:100D4000030100000000000000000000000000009F
:100D5000000000000000FF1F05001077407F4100E9
:100D6000417F001109650911004448534844003E81
:100D70000008142200221408003E0049494949494C
:100D8000005C5653565C0007017740400004077131
:100D90004040007F515D457F00FF0000000000FFE4
:100DA00008080808080808080808FF08080F0F08BE
:100DB000080304081020408080808080804020103C
:100DC0000804030808080808080000FFFF00008066
:100DD000C0E0F0F8F8F8F8F8F8F8F8F8F8F0E0C043
:100DE000800102FCF800000000000000000000008C
:100DF00000000000000000000000000000000000F3
:100E000000000000000000000000000000000000E2
:100E1000000000000000FF554055005500415549B5
:100E200055410041495D4941004149494941005D01
:100E300049415D4900495D41495D00415D5D5D415C
:100E400000417F5D4941007F415D49417F000000D5
:100E500000000000000000000010034D0079005366
:100E6000004B0065006500620000000A0344004179
:100E7000004700330000000403090409023B00029C
:100E80000100A0FA09040000010301010009211179
:100E90000100012240000705810308000109040147
:100EA000000103000000092111010001226D00076B
:100EB0000582032000011201000200000008EDFE7F
:100EC000606000010102000105010980A1018503A4
:100ED00019012AB700150126B70095017510810088
:100EE000C0050C0901A101850419012AA002150100
:100EF00026A002950175108100C005010906A10117
:100F00008506050719E029E71500250195087501F3
:100F100081020507190029EF1500250195F07501DB
:100F200081020508190129059505750191029501B0
:100F300075039101C005010906A101050719E02902
:100F4000E715002501950875018102950175088155
:100F5000010507190029FF150026FF0095067508F1
:100F60008100050819012905950575019102950172
:100F700075039101C00011241FBECFEFDAE0DEBF80
:100F8000CDBF12E0A0E0B1E0E4EDFFE502C00590C6
:100F90000D92A231B107D9F727E0A2E1B2E001C07A
:100FA0001D92A93BB207E1F70E94DF1C0C94E82FC9
:100FB0000C940000FC018081813069F481858823D4
:100FC00019F085E392E005C082858111FACF8FE1A7
:100FD00092E00C94C9090895FC018081813019F4D4
:100FE00086E292E009C0823019F48FE20C94F50B8E
:100FF000833021F48FE292E00C94C9090895FC013A
:101000008081813019F487E292E009C0823019F4BE
:1010100080E30C94F50B833021F480E392E00C9490
:10102000C9090895FC018081813079F48185882384
:1010300011F084E308C082858111FBCF84E392E044
:101040000E94C9098CE20C94F50B089561E074E0EC
:1010500080E591E00C94981ECF93C82F60E08EE459
:1010600091E00E94861E60E08CE491E00E94861E62
:101070008C2F827261E009F460E088E491E00E94C4
:10108000861E60E086E491E00E94861E61E08C2F5F
:10109000817109F460E082E491E00E94861E60E0C4
:1010A00080E491E00E94861E61E08C2F887809F42C
:1010B00060E08CE391E00E94861E60E08AE391E0AC
:1010C0000E94861EC47461E009F460E086E391E04A
:1010D0000E94861E60E084E391E00E94861E60E02C
:1010E00082E391E0CF910C94861E60914C02709146
:1010F0004D0280914E0290914F020E94A40A8130CD
:1011000069F040F0823071F0833081F460E08EE06D
:1011100091E00FC060E089E291E00BC060E080E206
:1011200091E007C060E087E191E003C060E084E007
:1011300091E00C94861ECF93C82F60E082E091E08E
:101140000E94861EC0FD03C086EF90E002C08CEFB7
:1011500090E060E00E94861E60E084EF90E00E94D4
:10116000861EC1FD03C088EE90E002C08EEE90E0C6
:1011700060E00E94861E60E086EE90E00E94861E7F
:10118000C2FD03C08AED90E002C080EE90E060E016
:101190000E94861E60E088ED90E0CF910C94861E40
:1011A0009C013056211540E2340748F0305E21158D
:1011B00040E1340720F0315C21153F4110F49927BC
:1011C00006C08F3F910519F010F080E090E0EBE150
:1011D000F2E02291218322E0E431F207D1F78F3F40
:1011E000910531F0FC01EF57F84F84918093140280
:1011F0000895CF93DF93FB012281222331F0EC018C
:101200000E945228CE010E94D00881E0DF91CF9148
:10121000089560E084E192E00C946A1E82E00895F3
:10122000CF930E942420882309F44EC00E949E1A66
:10123000882309F447C060E089EC98E00E94861E8C
:101240000E94750860E086EC98E00E94861E0E946D
:10125000090962E084E10E948D1D60E084EC98E061
:101260000E94861E60E08EEA98E00E94861E60E082
:101270008CEA98E00E94861E0E94DB260E949B0852
:1012800060E084EC98E00E94861E60E086E998E0C9
:101290000E94861E60E08CEA98E00E94861E0E94F2
:1012A000F313C82F0E9419148C2B0E942C0860E0A5
:1012B00084EC98E00E94861E60E080E898E00E943E
:1012C000861E02C00E94260880E0CF9108959C01EE
:1012D0003A9521153F4130F5BC0166277270AC018B
:1012E000442754709C012227387094FF0FC090FF50
:1012F00002C080E101C080E0672B09F08062452BCD
:1013000009F08064232B79F080680895892F81701B
:10131000672B09F08260452B09F08460232B19F0BC
:101320008860089580E00895CF93DF93EB010E94D9
:101330006709FE01DF91CF910994CF93DF93EC0110
:10134000805E9109089710F0209719F46EEF7BE00A
:1013500002C06EE77EE0CE010E9494098C2FDF91DF
:10136000CF910C94640BCF93DF93EC010E94B20BEE
:10137000CE01805E9109089710F0209719F465E07E
:101380007CE002C065E87EE0CE01DF91CF910C9455
:101390009409CF93DF93EC010E949D09C933D105D5
:1013A00049F42FEF87EE93E0215080409040E1F721
:1013B00000C00000CE01DF91CF910C94B30981E011
:1013C00008950C94F90808950C94E3091F93CF93A2
:1013D000DF9300D000D01F92CDB7DEB749835A8388
:1013E0006B8330911E0289819A81311114C066236A
:1013F00059F0222349F00E944D10182F682F89813F
:101400009A810E94F60F03C00E942110182F698153
:101410007A81812F04C00E944D1069817A810F90DA
:101420000F900F900F900F90DF91CF911F910C9420
:101430007C17FC01262F4081518162817381848158
:101440000C94E60981E00895CF93DF93EC0160E00E
:101450000E94190ABE01DF91CF910C94E4090C940B
:10146000E9180C94E51808950E94A00E0E94330A12
:101470002FEF84E39CE0215080409040E1F700C0D2
:1014800000000C94AF280F931F93CF93DF938C0130
:1014900061E00E94190AEC01B8010E940223B80120
:1014A000CE010E94E109882309F444C0B801CE01AD
:1014B0000E944D238823F1F1B801CE010E944E22F3
:1014C0008823C1F1B801CE010E946220882391F1E6
:1014D000B801CE010E94AA21882361F1F80182811E
:1014E000882309F1CB358DE5D807C1F050F4C1153B
:1014F000FCE5DF0781F0CF3DDC45A9F40E948115B2
:1015000019C0CC35EDE5DE0761F0CD35DD4559F488
:101510000E94CA1408C00E94340A0CC00E94D3144E
:1015200002C00E94D614C801DF91CF911F910F9184
:101530000C94DF0980E0DF91CF911F910F91089506
:101540000E94050B0C940D28CF92DF92EF92FF9230
:101550006C01EE24FF24C114D104E104F10421F054
:10156000C701B60120E101C020E0C72ED82EE92E28
:10157000FF24C114D104E104F10419F0285FC7016C
:10158000B6016B017C0154E0F694E794D794C794BC
:101590005A95D1F7C114D104E104F10419F02C5F7C
:1015A000C701B6016B017C0142E0F694E794D79441
:1015B000C7944A95D1F7C114D104E104F10419F09C
:1015C0002E5FC701B601DC01CB01B695A7959795B3
:1015D0008795892B8A2B8B2B09F02F5F822FFF9009
:1015E000EF90DF90CF90089508950C94F40A81E075
:1015F00008950C94F70A0895CF93C82F0E94F50A16
:101600008C2F0E94F90ACF9108950E94DB260C943A
:10161000FC0A0E94DB2690911D02891721F080931D
:101620001D020C94FC0A0895CF93DF93CDB7DEB76B
:101630002B970FB6F894DEBF0FBECDBF4F835887F0
:1016400069877A878B8761110E9416149E012F5F2C
:101650003F4F86E0F90111928A95E9F785E0FE0196
:101660003796D90101900D928A95E1F789819A8187
:101670004C815D81452B31F09F3F31F491E08F3FEC
:1016800019F403C091E001C090E090FF09C04981C6
:101690005A816B817C818D819E810E94341305C0AB
:1016A000C9010E94220A8111F2CF2B960FB6F8943D
:1016B000DEBF0FBECDBFDF91CF910895FC018081C9
:1016C00091810E948F100895CF93882309F448C018
:1016D000C82F8CEF8C0F813AD0F46C2F80915A0177
:1016E00090915B010E944A27882349F06C2F8091DA
:1016F0005A0190915B010E94D5270E9438146C2FEB
:1017000080915A0190915B010E94CA270CC080E22F
:101710008C0F883058F4C77081E001C0880FCA95DB
:10172000EAF70E94F613CF910C943814EBE5EC0F16
:10173000E33040F4F0E0E953FE4F808190E0CF9138
:101740000C940827C85AC73158F4EC2FF0E0EE0F7C
:10175000FF1FE756FE4F80819181CF910C941E2789
:10176000CF910895882349F1682F8CEF860F813A35
:1017700038F480915A0190915B010E94D5270CC0EA
:1017800080E2860F883050F4677081E001C0880FD6
:101790006A95EAF70E94FC130C9438148BE5860FC7
:1017A000833020F480E090E00C940827685A673179
:1017B00020F480E090E00C941E2708951F93CF93AF
:1017C000DF93182FEB010E94640B209741F08FE903
:1017D0009FE00197F1F700C000002197F6CF812F1D
:1017E000DF91CF911F910C94B20B893319F060E017
:1017F00070E002C060E570E00C94DE0B882321F0FD
:101800000E94F6130C9438140895882321F00E9446
:10181000FC130C9438140895CF92DF92EF92FF924C
:101820000F931F93CF93DF937C01D62FC72FFC011B
:101830001281058102950F700E94EC138823B9F084
:101840001123A9F08C2F807F803421F080E28D0F4E
:10185000883068F08091890382FD09C082E00E948F
:1018600098140E94EC1391E0D82ED92601C0D12CF7
:10187000CC2EC2948FE0C8228C2D90E08C30910544
:1018800008F0C4C1FC01EA5AFF4F0C94812F8C2F41
:10189000807FCF70882311F0C295C07F112399F00B
:1018A000CC2309F49FC180E28D0F883010F0D11154
:1018B00004C08C2F0E94F61303C08C2F0E940914C1
:1018C0000E9438148FC18D2F0E94B20BCC2309F4D3
:1018D0009DC180E28D0F883038F1DD2329F18C2FF6
:1018E0000E940F1424C08C2F807FCF70803211F0A3
:1018F000C295C07FDD2319F0D130A1F13DC08091A8
:10190000890382FF17C0112349F0CC2329F08C2FC3
:101910000E94F6130E94381480E065C180E00E94A6
:10192000B20BCC2309F472C18C2F0E94FC130E94CD
:1019300038146CC1112371F0002341F0013031F4EF
:101940000E9419148C2B0E94211460C10E9419144A
:101950008C2B1DC0002319F0013009F457C10E94DF
:101960002E1425C0112321F0063008F04FC10EC0FF
:10197000053008F04BC11BC0112361F0002331F08A
:10198000F701858180FF2EC18F7085838C2F0E9487
:10199000FE0B3CC1002359F0D93309F034C1FFEFED
:1019A00007EE13E0F15000401040E1F72AC18C2F00
:1019B0000E94050C2BC18C2F86958695837019F09B
:1019C000813061F023C1112321F08D2F9C2F937062
:1019D00002C080E090E00E94082720C1112321F07E
:1019E0008D2F9C2F937002C080E090E00E941E27F4
:1019F00015C18C2F837009F047C011110BC12D2F19
:101A0000229526952770220F220F6D2F6F70862F3B
:101A100090E0A0E0B0E0022E04C0880F991FAA1F3A
:101A2000BB1F0A94D2F7D4FF10C04FE050E060E033
:101A300070E004C0440F551F661F771F2A95D2F728
:101A4000409550956095709503C040E050E0BA0114
:101A5000C695C695C3708A019B01082B192B2A2BAA
:101A60003B2BC901B801C23049F058F4C13019F01C
:101A70000E940C0FCFC00E94FA0ECCC00E941E0F15
:101A8000C9C00E94F80EC6C0112319F08C2F8170B6
:101A900001C08695882309F4BDC02D2F2295269577
:101AA0002770220F220F6D2F6F70862F90E0A0E01D
:101AB000B0E0022E04C0880F991FAA1FBB1F0A9412
:101AC000D2F7D4FF10C04FE050E060E070E004C0F7
:101AD000440F551F661F771F2A95D2F740955095E2
:101AE0006095709503C040E050E0BA01C695C69578
:101AF000C3708A019B01082B192B2A2B3B2BC90190
:101B0000B801C23049F058F4C13019F00E94D10F29
:101B100081C00E94BF0F7EC00E94E30F7BC00E9465
:101B2000320F78C0CF70112339F08C2F0E94580FDC
:101B30008D2F0E94FE0B6EC08D2F0E94050C8C2FE6
:101B40000E94790F67C0D23F21F128F4D03F41F0C5
:101B5000D13FC1F043C0D33F19F1D43F79F03EC02B
:101B6000112341F0053008F051C08C2F8F710E9475
:101B70009E0F4CC0063008F049C0F7CF8091890312
:101B800082FF18C0112339F08C2F8F710E94580FDB
:101B90003DC01123C9F38C2F8F710E94790F36C07D
:101BA000112329F08C2F8F710E94430F2FC00E94A8
:101BB0003E0F2CC0112349F0CF718C2F0E94580F7B
:101BC00063E08C2F0E947D1421C081E00E94981454
:101BD0000230E0F082E00E94981418C0112331F026
:101BE000002391F28D2F0E94640B10C0002399F204
:101BF000D93349F41FEF27EE33E011502040304035
:101C0000E1F700C000008D2F0E94B20B88EF8C0D11
:101C1000843020F40E94DB260E94FC0ADD20C9F0FB
:101C20000E94E81380FD15C0F70112820E94E213A2
:101C30000E94580FC7010E944A0E0E94E213DF91D2
:101C4000CF911F910F91FF90EF90DF90CF900C9468
:101C5000790FDF91CF911F910F91FF90EF90DF905F
:101C6000CF9008950F931F93CF93DF93EC0168817A
:101C700079818A810E949A108C010E94F50F0E943E
:101C8000E60EB801CE010E940C0CDF91CF911F919E
:101C90000F910895CF93DF93EC01988189812B8177
:101CA0003C81232B31F08F3F31F481E09F3F19F4C9
:101CB00003C081E001C080E080FD1DC0CE010E9414
:101CC000430A811110C00E94EC138823A1F08A817D
:101CD000882389F08091890382FD0DC082E0DF9125
:101CE000CF910C949814CE010E94320ECE01DF9158
:101CF000CF910C94240ADF91CF910895882321F08D
:101D00000E9409140C9438140895882321F00E942D
:101D10000F140C943814089580E090E00E94082776
:101D200080E090E00E941E270E9416140C94381444
:101D300080915A0190915B010E94E0270C948C0ED7
:101D40000E9403140C94980E92959F70963079F02F
:101D500010F4925001C09A50923068F4803F69F0BC
:101D600018F4883E40F409C0843F29F406C0883E38
:101D700020F0813F11F080E0089581E00895FC019A
:101D8000808191810E948F100E94A40E0895CF93AC
:101D9000DF9300D000D01F92CDB7DEB70F900F9029
:101DA0000F900F900F90DF91CF910895CF93DF9315
:101DB00000D000D000D0CDB7DEB726960FB6F8948D
:101DC000DEBF0FBECDBFDF91CF9108950895089576
:101DD0000C94E70E0C94E80E0E94EA0E60935002F9
:101DE0007093510280935202909353020C948C0E84
:101DF0000C94EC0E0F931F9300915002109151021E
:101E00002091520230915302602B712B822B932B25
:101E10001F910F910C94EC0E0F931F9300915002A1
:101E2000109151022091520230915302602371238C
:101E3000822393231F910F910C94EC0E0F931F9309
:101E400000915002109151022091520230915302A0
:101E500060277127822793271F910F910C94EC0E16
:101E60000C94E70E0E94300F60934C0270934D0269
:101E700080934E0290934F020C948C0E60E070E0C1
:101E8000CB010C94320F0F931F9341E050E060E0C0
:101E900070E08A019B0104C0000F111F221F331F35
:101EA0008A95D2F7C901B8011F910F910C94320F96
:101EB0000F931F9341E050E060E070E004C0440FD6
:101EC000551F661F771F8A95D2F780914C0290911B
:101ED0004D02A0914E02B0914F028A019B01082B46
:101EE000192B2A2B3B2BC901B8011F910F910C9480
:101EF000320F0F931F9341E050E060E070E004C0A8
:101F0000440F551F661F771F8A95D2F7409550954D
:101F10006095709580914C0290914D02A0914E0277
:101F2000B0914F028A019B01082319232A233B23E6
:101F3000C901B8011F910F910C94320F0F931F9399
:101F400041E050E060E070E004C0440F551F661FA0
:101F5000771F8A95D2F780914C0290914D02A09103
:101F60004E02B0914F028A019B01082719272A27A8
:101F70003B27C901B8011F910F910C94320F0F93A9
:101F80001F9300914C0210914D0220914E0230910E
:101F90004F02602B712B822B932B1F910F910C946E
:101FA000320F0F931F9300914C0210914D0220911C
:101FB0004E0230914F0260237123822393231F919D
:101FC0000F910C94320F0F931F9300914C021091BC
:101FD0004D0220914E0230914F02602771278227D7
:101FE00093271F910F910C94320F089527E0929F31
:101FF000800D1124E82FE695E695E695877051E06F
:1020000001C0550F8A95EAF785E0E89FF001112499
:10201000E15EFD4F20E030E070E04081CB01022E18
:1020200002C0969587950A94E2F78170819584277E
:102030008523842781932F5F3F4F2530310569F732
:10204000089527E0929F800D1124682F669566956C
:102050006695982F977085E0689FB001112440E045
:1020600050E080E0FB01E40FF51FE15EFD4F2081B1
:1020700030E0092E02C0369527950A94E2F72170C8
:102080003327042E01C0220F0A94EAF7822B4F5FF8
:102090005F4F4530510531F70895BF92CF92DF92DF
:1020A000EF92FF920F931F93CF93DF938C01C09019
:1020B0004C02D0904D02E0904E02F0904F02809181
:1020C000500290915102A0915202B0915302C82A3D
:1020D000D92AEA2AFB2ACFE1D0E0D701C6010C2E8B
:1020E00004C0B695A795979587950A94D2F780FD79
:1020F00004C0219790F7B12C07C0BC2EB8018C2FDB
:102100000E948F170197A9F38B2DDF91CF911F911B
:102110000F91FF90EF90DF90CF90BF900895CF93F5
:10212000DF93EC010E944D10BE010E948F17DF91DA
:10213000CF9108951F93CF93DF93EB0190911E02EF
:10214000992321F0CB010E948F1013C0882349F0FE
:10215000CB010E944D10182F682FCE010E94F60F60
:1021600004C0CB010E942110182FBE01812F0E94B4
:102170008F17DF91CF911F9108951F93CF93DF9316
:10218000C091540216E080915502C81799F0D0E032
:102190001C9FF0011D9FF00D1124EA5AFD4F408154
:1021A000518162817381848195810E94D60E21962E
:1021B000C770E9CFDF91CF911F91089540918602BA
:1021C00050918702609188027091890280918A0201
:1021D00090918B020C94D60EEF92FF920F931F9367
:1021E000CF93DF9380918B0282958F7009F065C049
:1021F00080918802882309F460C080915402F09095
:1022000055021091860200918702609189027091B7
:102210008A0291E01F3F09F090E0C0915801D091EF
:102220005901292F96E0E92E8F1509F446C0611552
:10223000710521F00F3F21F030E003C031E001C013
:10224000322F90E030FD36C0E89EF001E99EF00D9F
:102250001124DF01AA5ABD4F11963C9111973013FA
:1022600029C03C91311326C012963C91129731112E
:1022700021C013964D915C911497461B570B4C1738
:102280005D07C0F480918B028F70806180938B0218
:10229000E55AFD4F80818F708061808386E892E0EF
:1022A0000E944A0EDF91CF911F910F91FF90EF9006
:1022B0000C94BD1001968770B7CFDF91CF911F911D
:1022C0000F91FF90EF9008959F92AF92BF92CF929F
:1022D000DF92EF92FF920F931F93CF93DF93CDB7CF
:1022E000DEB761970FB6F894DEBF0FBECDBF8C018D
:1022F00085E0F801DE011D9601900D928A95E1F7C7
:10230000D8011296EC9090918602E091870220917C
:10231000890230918A022115310531F0EF3F31F405
:1023200081E09F3F19F403C081E001C080E0B82F35
:10233000B1709B2E80FD47C1D8014C9111965C91E4
:1023400011971396AD90BC90149786E8C82E82E042
:10235000D82EF0908802B501621B730B20915801B2
:1023600030915901FF2009F4D9C080918B02621786
:10237000730708F095C0282F207F09F052C05E1324
:1023800013C0491311C0FE2CE1100EC08F70806184
:1023900080938B020E94DE10C6010E944A0E80913B
:1023A0008B02F80185834DC1AB2831F05F3F31F4DA
:1023B00081E04F3F19F403C081E001C080E080FD5F
:1023C00003C081E08E2502C080E090E0F82FF1701C
:1023D000FF2E80FF1CC0809154022091550236E0F0
:1023E000821709F40BC190E0389FF001399FF00D7E
:1023F0001124EA5AFD4F6181561306C060814613CD
:1024000003C06281E61203C001968770E9CFFE2CFB
:10241000EE2009F416C180918B02816080938B02BB
:1024200054C05E1306C0491304C0E11002C0F80195
:1024300099C0C8010E94BF0E882361F1EE2051F1BE
:1024400020918B02822F82958F7090E0029774F01A
:10245000809186029091870298878F831986BB8628
:10246000AA862C87CE0107960E944A0E86E0F801C4
:10247000A6E8B2E001900D928A95E1F70E94EC1077
:102480000E94DE100AC05E1711F1C8010E94BF0E43
:1024900081112CC0C8010E944A0EFF24F394D1C0C0
:1024A000282F207F81F77A2DB98AA88A6E2D8989F5
:1024B0000E94C70E86E892E00E944A0E86E0D6018E
:1024C0001D928A95E9F70E94DE10F12CBAC04913DB
:1024D000DCCFE110DACFF8018583C8010E944A0EF3
:1024E00086E0D6011D928A95E9F7ABC0EE2091F205
:1024F00020918B02822F82958F7090E002970CF4CE
:10250000B5CF80918602909187029A8389831B823E
:10251000BD82AC822E83CE010196A6CF62177307CF
:1025200008F044C0FE2CEE2009F4B4CF5E1330C096
:1025300049132EC020918B0220FD21C0822F82954D
:102540008F70482F50E041155105C9F0F8012583DF
:102550004F30510541F08F5F982F9295907F822FD9
:102560008F70892B8583C8010E944A0E86E0F8018E
:10257000A6E8B2E001900D928A95E1F73CC086E0B2
:10258000F801A6E8B2E001900D928A95E1F759C0F2
:10259000C8010E94BF0E811169CF80918B028160BA
:1025A00080938B02C8010E944A0E4BC07A2DB98AD3
:1025B000A88A6E2D89890E94C70E86E0D6011D92D9
:1025C0008A95E9F718C0EE2009F464CFC8010E948B
:1025D000BF0EF82E882309F45DCF86E0F801A6E847
:1025E000B2E001900D928A95E1F786E892E00E94B0
:1025F0005E0B0E94EC100E94DE1023C04D875E87A8
:102600008D859E850E948F10292F22952F70223054
:1026100028F49F7039F0811105C00BC0243028F4D4
:102620009F7049F4805E883020F0C8010E944A0EF5
:102630009F2CF92C06C0D80115969C91907F91F79C
:10264000F8CF8F2D61960FB6F894DEBF0FBECDBFC9
:10265000DF91CF911F910F91FF90EF90DF90CF907E
:10266000BF90AF909F9008951F93CF93DF93CDB706
:10267000DEB72C970FB6F894DEBF0FBECDBF4F83E9
:10268000588769877A878B879C87CE0107960E9437
:1026900064118823D1F09F8188852A853B85232B6F
:1026A00031F08F3F31F481E09F3F19F403C081E0A6
:1026B00001C080E080FD47C04F81588569857A85DB
:1026C0008B859C850E94D60E3EC086E0FE01379623
:1026D000DE01119601900D928A95E1F7FF81E88560
:1026E0006A857B856115710531F0EF3F31F481E03A
:1026F000FF3F19F403C081E001C080E080FD23C0EA
:102700002091550230E0C9010196877099274091C8
:10271000540250E084179507F1F1F983EA837D8331
:102720006C8396E0929FD001939FB00D1124AA5A1A
:10273000BD4FFE01319601900D929A95E1F780937D
:1027400055020E94BD1016E08091540290915502EE
:10275000891771F1189FC00111248A5A9D4F0E9458
:102760006411882329F1E09154021E9FF001112485
:10277000EA5AFD4F40815181628173818481958144
:102780000E94D60E8091540290E00196877099279E
:1027900080935402D9CF0E94A00E1092550210923D
:1027A0005402E6E8F2E086E0DF011D928A95E9F73F
:1027B0002C960FB6F894DEBF0FBECDBFDF91CF9140
:1027C0001F9108958091AC02859585958595089512
:1027D0008091AC02877008959091AC02977081E06F
:1027E00009F480E008958091CF0208959091CF027E
:1027F000892B8093CF02089580959091CF028923F1
:102800008093CF0208951092CF0208958091CE0256
:1028100008959091CE02892B8093CE0208958095E1
:102820009091CE0289238093CE0208951092CE0219
:1028300008958091AD02089508950C941C140C9491
:102840001D149091890392FD08C09091AD029817D4
:1028500021F08093AD020C941F1408958091AD0275
:10286000882329F01092AD0280E00C941F14089583
:10287000CF93DF93E0915A01F0915B018091CF02F9
:102880008083E0915A01F0915B0190818091CE02AA
:10289000892B80838091AD02882381F0E0915A01D9
:1028A000F0915B019081892B808380915A019091F6
:1028B0005B010E94342781110E942E14C0915A019D
:1028C000D0915B0140E250E06CE872E0CE010E94E2
:1028D000902F892B69F080E2FE01ACE8B2E0019014
:1028E0000D928A95E1F7CE01DF91CF910C94EE26FF
:1028F000DF91CF9108950C941C149091890392FD5F
:1029000010C098E0899F90011124262B2093AC02DF
:102910000E94580F8091AC028595859585950C9401
:102920007B140C94580F1092AC0280E00C947B1432
:102930002091AC02809582238093AC02982F9770EF
:1029400099F430E0482F082E000C550B241735075A
:1029500059F09091890392FD07C0859585958595DD
:102960000E94790F0C94931408959091890392FB1F
:10297000222720F9281769F080FB92F990938903A8
:1029800080918803909189030E94FD1482E00C9449
:10299000981408958091890382FB882780F991E03B
:1029A00089270C94B51481E00C94B51480E00C9444
:1029B000B51480E090E00E94AE2F21E0893E9E4F4A
:1029C00009F020E0822F089582E090E00C94A62F79
:1029D00083E090E00C94A62FCF9384E090E00E94D7
:1029E000A62FC82F82E290E00E94A62F2C2F30E065
:1029F000A901582BCA01CF910895CF93C92F682FF1
:102A000084E090E00E94B42F6C2F82E290E0CF919E
:102A10000C94B42FAB01BC018FE090E00C94C62F56
:102A2000AB01BC0183E190E00C94C62F60E070E044
:102A3000CB010C94101560E070E0CB010E940A15E8
:102A40000C94161569EE7EEF80E090E00E94D22F84
:102A500060E082E090E00E94B42F60E083E090E0CC
:102A60000E94B42F10925002109251021092520202
:102A70001092530260E084E090E00E94B42F60E086
:102A800082E290E00E94B42F60E085E090E00E9436
:102A9000B42F60E086E090E00E94B42F6FEF87E0F3
:102AA00090E00E94B42F40E050E0BA0188E090E04E
:102AB0000E94C62F60E08DE090E00E94B42F40E0BD
:102AC00050E0BA0188E190E00E94C62F60E087E103
:102AD00090E00E94B42F40E050E0BA018CE190E019
:102AE0000E94C62F60E070E080E290E00E94D22F4A
:102AF00040E050E0BA0188E190E00E94C62F0C94BB
:102B00001B150C9422158EE090E00E94A62F91E0F8
:102B1000811101C090E0892F0895682F8EE090E028
:102B20000C94B42F0E9452286093DE027093DF024F
:102B30008093E0029093E1026093DA027093DB02EB
:102B40008093DC029093DD02089585B7806885BF8D
:102B500085B7806885BF08950C949E1A08950C94DB
:102B6000AE150C94AE150C94B1150C94AE150C94D6
:102B7000B5150C94AE150E94A5158CEA98E10E943B
:102B8000D1260E94B9150C94B7150E94AF150C946C
:102B9000AE150E94AF180C94FB0A0E943D280E94BB
:102BA0006B180E94C11A0E94EE190E94C9150E945A
:102BB000EC1C80E00E94431D0E94CB1A0C94B315BC
:102BC0008F929F92AF92BF92CF92DF92EF92FF923D
:102BD0000F931F93CF93DF93CDB7DEB72A970FB62E
:102BE000F894DEBF0FBECDBF0E943A1A982E811115
:102BF0000E94921580EDA82E82E0B82E00E010E031
:102C0000802E802F0E94D318D82EF501C1905F012D
:102C1000C826B1F40F5F1F4F0A30110589F78FEFF7
:102C200089838A831B820E9446288160782F9D8336
:102C30008C8349815A816B818D810E94140B2FC036
:102C40008091E20281FD0E94D918E12CFF24F394C7
:102C50008C2D8F21F1F00E94AC15882399F0EE8223
:102C60008F82DF2081E009F480E088870E94462877
:102C70008160782F9A8789874E815F8168858A85F0
:102C80000E94140BF801E053FD4F8081F826F0827A
:102C900006C0E394FF0CF7E0EF12DACFBBCF81E080
:102CA000911001C080E02A960FB6F894DEBF0FBEE7
:102CB000CDBFDF91CF911F910F91FF90EF90DF90EB
:102CC000CF90BF90AF909F908F9008950E949E1AD2
:102CD00081110C94AA230895CF930E94E015C82F68
:102CE0000E9466160E942620C1110E94E51ECF9107
:102CF0000C94090BCF93DF930E949417EC0181157C
:102D000022E59207E8F5811531E5930708F0B6C092
:102D1000883E910528F5803E910508F0E9C0883A83
:102D2000910570F4853A910508F07AC081309105DB
:102D300009F473C008F4D9C0049708F0D9C0D5C00D
:102D40008F3B910508F0D1C0C85AD0E0CC0FDD1FF1
:102D5000C653DE4F0990D881C02DCE019464C9C0FE
:102D6000811540E5940708F069C0811550E4950786
:102D700008F060C09A9581159F4108F4B9C0B5C0AC
:102D8000811536E5930728F5811545E5940708F088
:102D900092C0811554E5950708F087C0AC014370D7
:102DA0005527282F26952695C115D34508F06CC0C8
:102DB00081E090E002C0880F991F4A95E2F740E257
:102DC000249F90011124EC01C22BD32BCE019C68CF
:102DD00090C081152AE5920780F4811539E59307A3
:102DE00008F072C0811548E5940708F47EC0D82F1A
:102DF000CC27CE01806F906A7CC09056811590429E
:102E000008F073C08D2F8F710E942818DD27D062C3
:102E10008F71AE01582BCA016CC081E090E069C08F
:102E2000C55AD0E0C850DE4F8881C82FD0E0CE010F
:102E300090645FC0DF70CE01906A5BC074E09695CD
:102E400087957A95E1F7282F23703C2F337081E026
:102E500090E002C0880F991F3A95E2F79C68AC0198
:102E6000522B9A019C2F9F709695969550E2959FB4
:102E7000E0011124C9018C2B9D2B3BC0D82FCC27FE
:102E8000CE01816F906A35C081E090E002C0880F6A
:102E9000991F4A95E2F750E2259F90011124EC0119
:102EA000C22BD32BCE019A6824C0D82FCC27CE01B9
:102EB000846F906A1EC00E9428188F7190E0D82FEE
:102EC000CC27CE01906215C08F700E94281894E024
:102ED000D695C7959A95E1F7CF70D0E0DC2FCC2737
:102EE000D0699E01282BC90104C080E090E001C098
:102EF000CE01DF91CF91089526E4829FC001112475
:102F0000FC0127E0729FE00DF11D1124E60FF11D79
:102F1000EE0FFF1FEF5AFA4F8591949108950E948A
:102F20007C170E947A1608958238910569F1B0F4F1
:102F30008133910509F46DC048F48932910509F493
:102F400063C08A32910509F469C0089585339105FB
:102F500009F455C089339105B9F00895833E910570
:102F600069F138F4803E9105B1F0823E910509F196
:102F70000895863E9105A9F1873E9105B9F1843EF9
:102F8000910509F064C023C02091880320FD4FC043
:102F900021FD4DC008958091880380FD44C080913B
:102FA000890380FF44C08091880384FD42C083EE82
:102FB0004DC08091880382FF38C0F5CF809188038F
:102FC00082FD33C08091890380FD31C0ECCF8091B8
:102FD000890381FF32C08091880384FD2AC087EE77
:102FE00035C08091880383FF26C0F5CF8091880388
:102FF00083FD21C08091890381FD1FC0ECCF8091AA
:10300000880385FD1CC01DC08091880385FD19C003
:1030100016C08091880386FD16C017C08091880372
:1030200086FD13C010C089E311C082EE0FC080EE90
:103030000DC080E00BC086EE09C084EE07C089E2B7
:1030400005C085E303C08AE201C081E390E00895F2
:103050009091880392FF0DC0282F2871283019F411
:10306000877F846006C0282F2471243011F48B7F61
:10307000886093FF0DC0282F2871283119F4877EAE
:10308000846106C0282F2471243111F48B7E88615D
:103090002091890320FF0DC0382F3871383019F482
:1030A000877F816006C0382F3171313011F48E7FF7
:1030B000886021FF0DC0282F2871283119F4877EE0
:1030C000816106C0282F2171213111F48E7E886123
:1030D00094FD877E089510928403109285031092C8
:1030E0008603109287030895CF92DF92EF92FF92AA
:1030F0006B017C010E949E1A81110EC00E94522811
:10310000C61AD70AE80AF90AC0928403D092850346
:10311000E0928603F0928703FF90EF90DF90CF90CC
:1031200008950F931F930E949E1A882321F01F91E8
:103130000F910C9452280E94522800918403109100
:1031400085032091860330918703600F711F821FD2
:10315000931F1F910F91089580E0089508950E9494
:10316000D914811102C00E9481150E94E414809339
:10317000E2020E94EC1490938903809388030E94DA
:10318000AE180E94E814682F70E080E090E00E9482
:10319000F80E60914C0270914D0280914E02909118
:1031A0004F020C94300FE82FF0E0EB56FC4F80817B
:1031B0000895089580EA8A95F1F7089500C008956A
:1031C0000C94DA1808950C94E2180C94E3180C94FB
:1031D000E2180C94E7180C94E218FF920F931F93D7
:1031E000CF93DF9300D000D01F92CDB7DEB70E94FF
:1031F0009E1A60919F038823E9F185E0F82E8E01E5
:103200000F5F1F4FF8018F2D11928A95E9F7862FD6
:1032100090E0B8018B569C4F0E94D91A882389F000
:1032200080918A0390E045E050E0B8018B569C4FB6
:103230000E94902F21E02093E302892B61F410E09B
:1032400016C08091E3028823D1F3F8011192FA9419
:10325000E9F71092E302A0918A03B0E0AB56BC4FAD
:1032600085E0F80101900D928A95E1F711E00E9446
:10327000310A0DC070E06B567C4F80918A0390E05C
:103280008B569C4F0E94631B0E94EB1810E0812F0D
:103290000F900F900F900F900F90DF91CF911F9193
:1032A0000F91FF900895F894E82FE295EF70F0E009
:1032B00031A1282F2F7081E090E001C0880F2A955E
:1032C000EAF7982F9095932391A392A1892B82A33B
:1032D000789408950F931F93CF93DF93CBEFD1E0B2
:1032E00089918F3F11F00E94531982E0C030D807B6
:1032F000B9F7CCE5D1E003E611E089918F3F11F0F9
:103300000E9453190C171D07C1F7DF91CF911F9130
:103310000F910895CF92DF92EF92FF920F931F9338
:10332000CF93DF938C01C62FD0E0CE0185509E4F06
:103330007C01FC0190819F3F09F447C0D62EF89490
:10334000E92FE295EF70F0E081A19F7021E030E07D
:1033500001C0220F9A95EAF7822B81A382A12095C2
:10336000282322A378940E94DE18ECE5F1E043E6DE
:1033700051E031E0C12C21912F3F89F0A22FA2957D
:10338000AF70B0E090968C9190E02F7002C0959550
:1033900087952A95E2F780FD02C0832F01C080E067
:1033A000C82A330F4E175F0731F7F70180818F3F2F
:1033B00011F00E94531961E0C11001C060E08D2D31
:1033C0000E94E018C00FD11FC882DF91CF911F91DA
:1033D0000F91FF90EF90DF90CF900895CF93DF9300
:1033E000CDB7DEB727970FB6F894DEBF0FBECDBFBF
:1033F00080916301811114C087E0E2E9F1E0DE0110
:10340000119601900D928A95E1F7FE013196ACE597
:10341000B1E0CE01089621912D93E817F907D9F76D
:1034200080916301811102C095E001C090E090930A
:103430009F0385E0891B80938A030E946A198AE0B2
:10344000E5E9F3E0DF01982F1D929A95E9F7EBE8A3
:10345000F3E0DF011D928A95E9F785E00E948E1A5C
:1034600027960FB6F894DEBF0FBECDBFDF91CF9188
:103470000C942F0AEF92FF920F931F93CF93DF9339
:10348000CDB7DEB72A970FB6F894DEBF0FBECDBF1B
:103490008E010F5F1F4F8AE0F80111928A95E9F7BC
:1034A000F12C6F2DC8010E948A19F394F5E0FF12E8
:1034B000F8CF4AE050E0B8018BE893E00E94902FEB
:1034C0007C0121E0892B09F420E0E114F10441F0B2
:1034D0008AE0F801ABE8B3E001900D928A95E1F73C
:1034E00060919F0370E06B567C4F45E08BE893E062
:1034F0000E948F1AEF2819F40E94ED1802C081E093
:1035000090E02A960FB6F894DEBF0FBECDBFDF91D4
:10351000CF911F910F91FF90EF9008950895FB01B7
:10352000DC0150E09D01281B390B241735071CF4E2
:103530002D912193F7CF08950C948315CF9380910B
:10354000E602811116C0C4E60E945B2F81110AC0F9
:103550008FE39CE90197F1F700C00000C150A1F78B
:1035600082E001C081E08093E602823011F40E9483
:10357000562F81E09091E602913009F080E0CF91E2
:1035800008950E949C1A809363010E949E1A8111E3
:103590000C94111B08950E949E1A811102C00C9474
:1035A000131B089581E09091E7029A3008F080E0C3
:1035B00008950F931F93CF93DF93EC018B018091BC
:1035C000E7028A3038F4B801CE010E94611B8111F4
:1035D0001DC00AC08091E4029091E5020E945E281D
:1035E000843F914080F715C08091E7028F3F19F02A
:1035F0008F5F8093E7028091E7028A3060F00E943B
:1036000046289093E5028093E40203C01092E702FB
:1036100002C080E001C081E0DF91CF911F910F9146
:1036200008950C946A250C946D25DF92EF92FF9219
:103630000F931F93CF93DF937901C82F880FDD0B72
:1036400041155105A9F0FE0193E0EE0FFF1F9A9579
:10365000E1F7EC59FE4F8181928188519D4F208185
:1036600030E04217530708F49A01A9010E949D2FE8
:10367000CE010E945626D82E8823D1F001151105BF
:10368000B9F083E0CC0FDD1F8A95E1F7FE01EC591C
:10369000FE4F438150E00417150708F4A801CC59E8
:1036A000DE4F6C817D8168517D4FC7010E949D2F47
:1036B0008D2DDF91CF911F910F91FF90EF90DF90B3
:1036C00008950C947D1C0C94991C0F931F93CF9319
:1036D000DF9300D000D0CDB7DEB76091FF027091CC
:1036E000000380910103909102030E946D286436CB
:1036F00071058105910528F10E949118DC01CB012B
:103700000296A11DB11D89839A83AB83BC8300E01F
:1037100010E020E030E044E050E0BE016F5F7F4FFA
:1037200082E00E94151B182F882361F00E94522806
:103730006093FF0270930003809301039093020350
:1037400001C011E0812F0F900F900F900F90DF912B
:10375000CF911F910F910895AF92BF92CF92DF92B8
:10376000EF92FF920F931F93CF93DF937C015B0146
:103770006A010E94D21A811103C001E010E002C068
:103780000AE010E0C1E0D0E0F894B501C701F6010D
:1037900009957894811115C021960C171D0794F096
:1037A000CC9F9001CD9F300D300D112480E090E032
:1037B00045E34A95F1F70000019682179307C1F798
:1037C000E3CF81E0DF91CF911F910F91FF90EF90B8
:1037D000DF90CF90BF90AF900895AF92BF92CF92FD
:1037E000DF92EF92FF920F931F93CF93DF9300D05E
:1037F00000D000D0CDB7DEB77B01C0900002D090E2
:10380000010201E010E09E012A5F3F4F40E050E0DE
:1038100060E070E080E00E94151B182F882309F4F7
:103820003EC056018FEFA81AB80A6091FB02709152
:10383000FC028091FD029091FE020E946D28643688
:1038400071058105910518F105E010E09E012F5FDB
:103850003F4F40E050E060E070E081E00E94151BC7
:10386000182F65E070E0C5010E94ED1C91E02E81EB
:10387000281390E0192339F10E9452286093FB022B
:103880007093FC028093FD029093FE0211C065E0EC
:1038900070E0C5010E94ED1C9E818913D5CF85E0A3
:1038A000F6013196DE01119601900D928A95E1F7AD
:1038B000112349F085E0FE013196A6EFB2E00190B8
:1038C0000D928A95E1F785E0E6EFF2E0D7010190ED
:1038D0000D928A95E1F7812F26960FB6F894DEBFF8
:1038E0000FBECDBFDF91CF911F910F91FF90EF9051
:1038F000DF90CF90BF90AF9008950F931F93CF9319
:10390000DF93EC018B014DEE5BE10E94AC1B882341
:1039100051F045E65BE1B801CE01DF91CF911F91F7
:103920000F910C94AC1B80E0DF91CF911F910F9110
:1039300008950F931F93CF93DF93F894C0910002E3
:10394000D0910102CE01019625E0FB01DC0101903E
:103950000D922A95E1F765E070E00E94ED1C8883E6
:103960007894F8946E817F81888599850091F20220
:103970001091F3022091F4023091F5026017710763
:103980008207930751F06093F2027093F3028093E1
:10399000F4029093F5020E9474187894DF91CF910D
:1039A0001F910F9108950E944B2A0E94CD150C94EF
:1039B000572A0E945B2A0E946C160C945C2A0E9473
:1039C0000F280E94322A0E94BB150E94D31C0E941D
:1039D000D91C0E94C515FBCF0895FC01680F791F03
:1039E0008FEF91E3E617F70771F02191822728E026
:1039F00030E087FF03C0880F892701C0880F21505E
:103A00003109B9F7EFCF0895EF92FF920F931F930B
:103A1000CF93DF93EC017B0164E670E088E70E94BE
:103A200004248C01EC0EFD1ECE15DF0561F017FDA0
:103A30000AC0FE01849164E670E00E9485248C0136
:103A40002196892B89F30E940925C801DF91CF9126
:103A50001F910F91FF90EF9008950895E0EAF3E031
:103A600080E094E0DF019C011D9221503040E1F79D
:103A7000F093A707E093A6078FEF9FEF90934F0374
:103A800080934E0308950E940E090E942D1D80937D
:103A90004A0380FD02C080E801C080E480934903AE
:103AA0000E94FE236DE070E08CE099E00E94041D0E
:103AB000892B11F080E0089580914A0363E070E063
:103AC00081FD03C089E099E002C086E099E00E9490
:103AD000041D892B79F76DE070E089EF98E00E9472
:103AE000041D892B39F70E945228DC01CB01805A32
:103AF0009541AF4FBF4F8093A2079093A307A09328
:103B0000A407B093A5070E942E1D81E080934D036A
:103B100080934C0310924B0308952091490336E0A3
:103B2000839FC0011124629F800D911D1124811576
:103B300024E0920714F080E090E080569C4F909330
:103B4000A7078093A60708952091A6073091A7079D
:103B50002A59334040914903642F70E0C9010E9403
:103B60006D2F481B463010F4240F311D211584E0C1
:103B7000380710F020E030E020563C4F3093A70784
:103B80002093A6070895CF93DF938A3011F481E044
:103B900003C08D3029F480E0DF91CF910C94391E61
:103BA000C62F682F8091A6079091A70726E0FC01F9
:103BB000A3E0B3E001900D922A95E1F7603E30F06A
:103BC00026E0FC0111922A95E9F70AC0F6E06F9F02
:103BD000B0011124675E764F46E050E00E94872FC7
:103BE000C11135C0C091A607D091A70746E050E0AB
:103BF000BE0183E093E00E94902F892BB1F1C05A5F
:103C0000D3409E0186E0369527958A95E1F781E0BD
:103C100090E0AC0102C0440F551F2A95E2F72091B5
:103C20004E0330914F03242B352B259646E0D69535
:103C3000C7954A95E1F702C0880F991FCA95E2F728
:103C4000822B932B90934F0380934E030EC0E091F1
:103C5000A607F091A7079F012A5F3F4F2E173F0746
:103C600009F2808180958193F9CFDF91CF910C94F7
:103C7000A41DCF93E82F2091A6073091A707205AC3
:103C8000334040914903642F70E0C9010E946D2FB9
:103C9000481B842FEE2359F066E00E94612FC82F45
:103CA000C150B0F060E080E20E94C31DF9CFA901CD
:103CB000480F511D4115544018F080E020E030E0DD
:103CC000280F311D20563C4F3093A7072093A6079D
:103CD000CF910895FF920F931F93CF93DF93EC0141
:103CE000F62EFC0101900020E9F78F010150110927
:103CF000C017D10728F46F2D89910E94C31DF8CFFA
:103D0000DF91CF911F910F91FF9008951F93CF9353
:103D1000DF93EC01162FFE018491882329F0612F97
:103D20000E94C31D2196F7CFDF91CF911F91089577
:103D3000EF92FF920F931F93CF93DF932091A607EB
:103D40003091A707205A3340A901460F571F413031
:103D5000544020F060E074E0621B730BC0914E038E
:103D6000D0914F03D901A056BC4FA901620F731F18
:103D700001E010E046175707E8F4FA01E21BF30BE5
:103D8000E80FF91FE491FC91EF1781F0EC93FA0131
:103D9000689415F8F695E7951694E1F7780102C056
:103DA000EE0CFF1CEA95E2F7CE29DF294F5F5F4F4B
:103DB0001196E0CFD0934F03C0934E03DF91CF9184
:103DC0001F910F91FF90EF90089580914D038823EC
:103DD000F9F00E945228DC01CB01805A9541AF4F87
:103DE000BF4F8093A2079093A307A093A407B0931B
:103DF000A50780914C0381110BC062E070E087EF52
:103E000098E00E94041D892B19F481E080934C03F3
:103E100080914C0308956F927F928F929F92AF9200
:103E2000BF92CF92DF92EF92FF920F931F93CF93A7
:103E3000DF9380914D03882309F4DDC020914E0368
:103E400030914F032115310509F4D5C080914B0302
:103E50008111D1C061E070E0082F10E03B01082E15
:103E600002C0660C771C0A94E2F7A901462157218B
:103E7000452B11F48F5FF0CF90914A03980166E0D3
:103E8000220F331F6A95E1F790FD13C08295880FCA
:103E9000880F807480937E01220F232F221F330B03
:103EA000319520938101815C80937F011092820182
:103EB00012C046E0369527954A95E1F7220F220F6A
:103EC000220F20937E0110928101295F20937F01B0
:103ED00087E08093820124E630E047E050E06CE721
:103EE00071E088E70E94B524892B09F084C0809195
:103EF0004A0380FD23C0A80196E0440F551F9A9500
:103F0000E1F740565C4F04E610E020E430E060E466
:103F100088E70E94DC24892B09F06DC00E94E51E11
:103F2000E301C095D09580914E0390914F03C82333
:103F3000D923D0934F03C0934E035DC080E4E9E0E2
:103F4000F3E0DF011D928A95E9F786E0000F111F6B
:103F50008A95E1F7AAE0B2E042E052E09924939416
:103F60002D91EA018991AE01B801680F711D60566B
:103F70007C4F30E0275F3C4FF90197E07F01E21A68
:103F8000F30AA92C01C0AA0CEA94EAF77B01B12C30
:103F9000E70189917E018A21892E8B18D82DD7704F
:103FA000CD2E0D2E000CDD08C82F01C0CC0FDA95E8
:103FB000EAF7D194C194D108D7E0CD22DD2401C025
:103FC0008695CA94EAF78C2BD0808D298083B39490
:103FD00088E0B812DDCF915031969F3F79F6C2E06C
:103FE000A231BC0709F0BCCF04E610E020E430E0C9
:103FF00049E053E08CCFDF91CF911F910F91FF905B
:10400000EF90DF90CF90BF90AF909F908F907F9078
:104010006F90089580914D0390914C03882389F00F
:10402000992369F062E070E085EF98E00E94041D3A
:10403000892B19F080914C03089510924C039091B4
:104040004C0381E08927089581E008950F931F9321
:1040500080914D03882399F18091A0079091A10749
:104060000E945E28C29760F00E9446289093A107A4
:104070008093A00760E080E00E948D1D0E941009DF
:104080000E940B1F80914C038823C9F00E94522884
:104090000091A2071091A3072091A4073091A507D2
:1040A000DC01CB01801B910BA20BB30B8F3F9F4F09
:1040B000AF4FBF4720F41F910F910C940A201F911E
:1040C0000F910895CF93DF93EC01FB018281882348
:1040D00009F43CC1C430FDE5DF0760F4CB3F9CE54B
:1040E000D90788F49E0122503C452431310508F05F
:1040F0002EC109C0C236EDE5DE0729F0C63AFDE55E
:10410000DF0709F024C10E94EC1490938903809387
:104110008803C1318CE5D80709F4C6C008F042C055
:10412000C930ECE5DE0709F49BC000F5C5308CE52D
:10413000D80709F485C078F4C330ECE5DE0709F44C
:1041400078C008F07AC0C230DC4509F0F5C0809133
:1041500088038160EFC0C7309CE5D90709F478C0B7
:1041600008F07AC0809188038061E4C0CD30FCE51E
:10417000DF0709F487C058F4CB309CE5D90709F470
:1041800079C008F07BC08091880388606FC0CF3011
:10419000FCE5DF0709F480C008F082C08091880345
:1041A000877FC8C0CE3F9CE5D90709F471C000F5F0
:1041B000C531FCE5DF0709F485C068F4C3319CE52F
:1041C000D90709F475C008F095C00E94A00E80912F
:1041D00088038F77AFC0CC3FFCE5DF07A9F108F07B
:1041E00054C0CB3FDC4509F0A7C08091890340C093
:1041F000C230EDE5DE0709F489C058F4C1158DE53C
:10420000D80709F45AC008F069C080918903826018
:104210002FC0C236EDE5DE0709F47CC0C63AFDE5E5
:10422000DF0709F481C0C330DD4509F085C080E0B7
:104230006EC08091880382607DC08091880316C023
:1042400080918803886076C08091890382604FC026
:104250008091880380626EC08091880380646AC008
:104260000E94A00E80918803806864C0846062C050
:1042700081603DC0809188038E7F5CC080918803FF
:104280008D7F58C08091880316C08091890318C023
:10429000809189038D7F2BC0809188038F7E4AC0D7
:1042A000809188038F7D46C0809188038F7B42C0B8
:1042B00080918803877F8B7F3DC0809189038D7FAC
:1042C0008E7F15C08091880382FB222720F991E020
:1042D000922790FB82F990FB83F92CC0809189038F
:1042E000982F909591708E7F892B90FB81F9809308
:1042F000890322C00E94A00E8091880387FB222799
:1043000020F991E0922790FB87F914C081E00E9488
:104310008D1512C08091880384FB222720F991E03B
:10432000922790FB84F906C080918803982F90957E
:1043300090FB80F980938803809188039091890392
:104340000E94FD140E94A00E80E001C081E0DF9178
:10435000CF910895CF93DF9386319C4541F5EB01D2
:104360000E94F313982F8A8120915A0130915B01AA
:10437000882379F09A7A81E009F480E080935003F1
:10438000911102C069E201C065E3C9010E94CA2718
:104390000AC080915003811102C069E201C065E347
:1043A000C9010E94D5270E94381480E001C081E035
:1043B000DF91CF9108950F931F93CF93DF93C42F75
:1043C000D22FFC0182818823C9F0409353030E94BD
:1043D0004628909352038093510380E28C0F8830DB
:1043E00008F057C0C77081E001C0880FCA95EAF78E
:1043F000DF91CF911F910F910C94FE0B809153038D
:10440000481330C080915103909152030E945E285E
:10441000883C910538F510E21D0FCD17B9F080E208
:104420008C0F883040F4C77081E001C0880FCA95B6
:10443000EAF70E94050C183028F581E09D2F97704F
:1044400001C0880F9A95EAF70E94FE0B802F0E9408
:10445000F50B1830F0F4D77081E001C0880FDA95C1
:10446000EAF70AC080E28C0F883098F4C77081E0C8
:1044700001C0880FCA95EAF7DF91CF911F910F9184
:104480000C94050C802FDF91CF911F910F910C940C
:10449000F50BDF91CF911F910F9108950F939C0120
:1044A000CB01243F4CE5340731F188F4293DFCE58C
:1044B0003F07D9F02A3D4CE5340779F1283D3C45CA
:1044C000A9F506E221EE41EE68ED7CE52BC0263F22
:1044D000FCE53F07E1F0A8F0273F3C4539F507E24E
:1044E00025EE46EE67EF7CE51DC007E225EE45EEC2
:1044F00069ED7CE517C006E221EE40EE64EF7CE555
:1045000011C007E225EE44EE65EF7CE50BC006E244
:1045100021EE42EE66EF7CE505C008E221E045EEC3
:104520006AED7CE50E94DB2180E008C0FC0182810D
:10453000882319F01092530301C081E00F91089570
:10454000CF93DF93EC0181E0898B8F810E94F6137A
:1045500088850E9409140E943814EA81FB81CE01EB
:104560000696309729F06C897D89DF91CF91099467
:10457000DF91CF910895EF92FF920F931F93CF9306
:10458000DF93FC012285211136C0EC01E380F48029
:10459000F7E5FF1A26E12E9DC0012F9D900D1124F5
:1045A000DC01A050BF4F1496ED91FC9115978A5FE6
:1045B0009E4F309729F054966D917C9155970995AF
:1045C00086E18E9D80018F9D100D112400501F4F9C
:1045D000F80187810E94FC13F80180850E940F1466
:1045E0000E943814188219861B861E821D82109222
:1045F000550310925403DF91CF911F910F91FF90BB
:10460000EF900895DF92EF92FF920F931F93CF9355
:10461000DF93FB0122812223C1F12091830130919C
:1046200084012F3F3F4F89F18C01C0E0D1E0E12CA4
:10463000F12CDD24D39480918301909184018E1517
:104640009F051CF18E818823D9F089859A85801772
:10465000910739F480915403909155030817190775
:1046600079F0DF861C870B878989811103C0CE0111
:104670000E94A022CE0106960E94BB220E94161420
:104680004FEFE41AF40A6696D6CFDF91CF911F91CF
:104690000F91FF90EF90DF900895EF92FF920F93AC
:1046A0001F93CF93DF939C0137552F3F310511F0B6
:1046B00008F048C04091830150918401421753078C
:1046C00024F43093840120938301FB017C018281D7
:1046D00096E1929F8001939F100D1124E801C05034
:1046E000DF4F888B92818E81992311F1FA86E986BA
:1046F0008F5F8E830E9446289E878D870E941914A3
:104700008F830E94F31388870E9406149885892B53
:104710008887E881F981C8018A5F9E4F309719F038
:104720006C897D890995F0925503E09254030AC083
:10473000882341F08989882329F0C8018A5F9E4F28
:104740000E94BB2281E0DF91CF911F910F91FF90DA
:10475000EF900895CF92DF92EF92FF920F931F9305
:10476000CF93DF9380918301909184010196E9F1C9
:10477000F12C96E1E92E0F2D10E0809183019091AC
:104780008401801791078CF1E09EF001E19EF00D0D
:104790001124E050FF4FC288D388C114D10419F40A
:1047A00088ECC82ED12CE09EE001E19ED00D1124B2
:1047B000C050DF4F8E818823B1F08D859E850E9489
:1047C0005E28C816D90678F48989811103C0CE0104
:1047D0000E94A022E09EC001E19E900D11248A5FFC
:1047E0009E4F0E94BB22F394C6CFDF91CF911F91C1
:1047F0000F91FF90EF90DF90CF9008951092B90045
:104800008CE08093B80008959F92AF92BF92CF92B0
:10481000DF92EF92FF920F931F93CF93DF93B82E07
:10482000EB010E9446286C01C431D10558F0CF3FFE
:104830008FEFD80759F0CE0164E170E00E946D2F30
:104840007B0107C0EE24E394F12C03C025E0E22EA7
:10485000F12C84E8A82E94EA992E1092BC00909234
:10486000BC000E9446288C018091BC0087FD08C0D6
:104870000E944628801B910B8E159F05A8F32AC025
:104880008091B900887F883041F08091B900887F9D
:10489000803119F00FEF1FEF1FC0B092BB00A09244
:1048A000BC000E9446288C018091BC0087FD08C096
:1048B0000E944628801B910B8E159F05A8F30AC005
:1048C0008091B900887F883111F0803419F700E0B9
:1048D00010E00EC00EEF1FEFCF3F8FEFD80709F4A7
:1048E000BCCFC6010E945E288C179D0708F4B5CF87
:1048F000C801DF91CF911F910F91FF90EF90DF9052
:10490000CF90BF90AF909F9008950F931F93CF9338
:10491000DF93EB018093BB0084E88093BC000E948E
:1049200046288C018091BC0087FD0EC0CF3F8FEFE1
:10493000D807C1F30E944628801B910B8C179D0756
:1049400088F38EEF9FEF0CC02091B900287F81E0A3
:1049500090E0283211F480E090E0919581959109E2
:10496000DF91CF911F910F910895CF92DF92EF9237
:10497000FF920F931F93CF93DF936B018A0179010D
:10498000B9010E940424E6010C0D1D1DC017D107BA
:1049900061F424E92093BC00DF91CF911F910F9126
:1049A000FF90EF90DF90CF90089597FDF2CFB70181
:1049B00089910E948524EACFCF92DF92EF92FF92F5
:1049C0000F931F93CF93DF93C62F6A017901B8012C
:1049D0000E94042497FD11C0B8018C2F0E948524E9
:1049E000E601EC0CFD1CCE15DF0539F097FD05C086
:1049F000B80189910E948524F6CF24E92093BC0058
:104A0000DF91CF911F910F91FF90EF90DF90CF90AA
:104A1000089584E98093BC0008958EE14B9B02C009
:104A20008150E1F74B9BFECF08955B9880E28A9519
:104A3000F1F75B9A0895FC012AE02A95F1F728E046
:104A400090E080E031E040E14A95F1F7880F4B9B20
:104A500002C08160932700C0000040E14A95F1F751
:104A6000215089F720E12A95F1F729B100C0000013
:104A700030E13A95F1F723FB222720F99227208194
:104A8000920F90830895EF92FF920F931F93CF930D
:104A9000DF931F92CDB7DEB719828C017C01E60E41
:104AA000F11C0E151F0551F00E940D25CE01019637
:104AB0000E941B25F80181938F01F3CF81E099813A
:104AC000911180E00F90DF91CF911F910F91FF9096
:104AD000EF900895539A5B9A089553985B9AEB9AD6
:104AE000E9E6F0E080818F7380830895615091E062
:104AF00001C0990F6A95EAF720E031E0992361F04F
:104B0000492F482319F05B9A232701C05B9840E2A4
:104B10004A95F1F79695F2CF222311F05B9A01C0E6
:104B20005B9880E28A95F1F75B980895FF920F9366
:104B30001F93CF93DF93EC018C01060F111DC0175B
:104B4000D10741F0F9900E94152568E08F2D0E9451
:104B50007625F5CFDF91CF911F910F91FF900895AA
:104B60001F920F920FB60F9211240F931F932F9342
:104B70003F934F935F936F937F938F939F93AF93E5
:104B8000BF93EF93FF93CF93DF931F92CDB7DEB721
:104B900019820E940D25CE0101960E941B25082F27
:104BA000069506950695902F96959570202F257061
:104BB000920F292F237096959695920F87708913DF
:104BC0005FC0898181115CC0043008F059C080E168
:104BD0008A95F1F75B9A539A82E08A95F1F700C0C3
:104BE0005B9888E0089F80011124D801AC59BE4F22
:104BF0001696ED91FC9117973097A9F060910002FD
:104C00007091010214962D913C911597260F371F34
:104C100011968D919C911297680F791F13964C9164
:104C200013978C910995F801EC59FE4F6381662327
:104C300051F0809100029091010224813581820F10
:104C4000931F0E9496250E94152580E18A95F1F711
:104C50005B9853985B9A80E18A95F1F7F801EC59DB
:104C6000FE4F6081662351F0809100029091010215
:104C700021813281820F931F0E9443250E940D25BE
:104C80000F90DF91CF91FF91EF91BF91AF919F91E5
:104C90008F917F916F915F914F913F912F911F91D4
:104CA0000F910F900FBE0F901F9018950F931F93A9
:104CB000CF93DF93843091050CF06DC0EC01F89434
:104CC000539A5B9885E08A95F1F700009C2F9695A2
:104CD00095702C2F2570920F892F8370969596953D
:104CE00023E0CC0FDD1F2A95E1F7980F8E01092BE9
:104CF0000E94152584E08A95F1F700C068E0802FB6
:104D00000E94762580E18A95F1F753985B9A4B993A
:104D100002C000C0FCCF87E090E04B9B08C0019729
:104D200021F4539A5B9A789436C000C0F6CFFE0106
:104D3000EC59FE4F6381662381F0809100029091CF
:104D4000010224813581820F931F0E944325811126
:104D500004C0539A5B9A78941FC00E940D2580E28C
:104D60008A95F1F75B98539A80E18A95F1F7CC59CF
:104D7000DE4F6881662351F080910002909101021C
:104D800029813A81820F931F0E9496250E94152542
:104D9000789481E001C080E0DF91CF911F910F9165
:104DA00008959093130280931202089590935C03E8
:104DB00080935B0308950E949E1A811103C0809125
:104DC00056030895E0915B03F0915C03309721F066
:104DD0000190F081E02D099480E00895E0915B035B
:104DE000F0915C03309799F020919101222359F0C2
:104DF0002091880327FF07C0DC012C9111962C938A
:104E0000119726E02C930280F381E02D09940895F8
:104E10002091590330915A032817390771F0909364
:104E20005A0380935903E0915B03F0915C03309740
:104E300021F00680F781E02D099408952091570311
:104E4000309158032817390771F0909358038093D5
:104E50005703E0915B03F0915C03309721F00084ED
:104E6000F185E02D09940895FC013296809191011D
:104E7000882331F08091880387FF02C09EE101C042
:104E800096E080E0915028F021912223D9F38F5FA2
:104E9000F9CF0895662351F1209191012223E9F081
:104EA0002091880327FF19C0462F469546954695C1
:104EB0004E31E0F4677021E030E002C0220F331F72
:104EC0006A95E2F7FC01E40FF11D828190E028234E
:104ED000392381E0232B69F409C0FC01329608963E
:104EE0002191621729F0E817F907D1F780E00895BA
:104EF00081E008959C01FC0132969FEF80E0419192
:104F0000461789F09F3F19F4411101C0982F8F5F18
:104F10008630A9F79F3F39F0F901E90FF11D97FDA0
:104F2000FA956283089508959C012A5F3F4FFC0122
:104F30004281461301C01282019682179307B9F786
:104F40000895262F2695269526952E3168F4FC0186
:104F5000E20FF11D677021E030E001C0220F6A9579
:104F6000EAF78281282B22830895262F26952695FD
:104F700026952E3170F4FC01E20FF11D677021E0DF
:104F800030E001C0220F6A95EAF72095828128233C
:104F90002283089520919101222329F020918803F2
:104FA00027FD0C94A1270C947A27209191012223AC
:104FB00029F02091880327FD0C94B5270C949427A1
:104FC00020919101FC013296222331F080918803D7
:104FD00087FF02C08EE101C086E0DF011D928A9545
:104FE000E9F7089508950C94F22783E080935D0318
:104FF0000C94F327811102C081E001C082E080930C
:105000005D030C94F3270C94FA2781E080935D03F1
:105010000C94F3270C94052808950C940C280895FB
:105020001F920F920FB60F9211248F939F93AF93FD
:10503000BF9380915E03811113C08091A807909166
:10504000A907A091AA07B091AB074196A11DB11D78
:105050008093A8079093A907A093AA07B093AB07E2
:10506000BF91AF919F918F910F900FBE0F901F90A6
:1050700018950E94A00E0C94A00A82E084BD93E0D3
:1050800095BD9AEF97BD80936E0008952FB7F89461
:105090008091A8079091A907A091AA07B091AB07AA
:1050A0002FBF08952FB7F8946091A8077091A907B2
:1050B0008091AA079091AB072FBF08959C014FB72D
:1050C000F8948091A8079091A907A091AA07B091A0
:1050D000AB074FBF821B930B0895CF92DF92EF92E5
:1050E000FF922FB7F894C090A807D090A907E0903E
:1050F000AA07F090AB072FBFA7019601261B370B1D
:10510000480B590BCA01B901FF90EF90DF90CF9087
:10511000089578941F920F920FB60F9211248F93D7
:105120009F93AF93BF938091A8079091A907A091F7
:10513000AA07B091AB070196A11DB11D8093A807E6
:105140009093A907A093AA07B093AB07BF91AF9123
:105150009F918F910F900FBE0F901F90189587E72A
:1051600097E790930108809300089AE088E10FB6D2
:10517000F894A895809360000FBE90936000FFCFD5
:105180008091820308950895CF93DF932091910138
:10519000222339F02091880327FF03C060E222E038
:1051A00002C068E021E02093E9002FEF3091E80091
:1051B000215035FD06C035ED3A95F1F7000021117B
:1051C000F5CF2091E80025FF1DC0EC0180919101F1
:1051D000811105C040E050E068E070E003C070E07D
:1051E00040E050E0CE010E94B82A8091E8008E771E
:1051F0008093E80080E2FE01A2E6B3E001900D9208
:105200008A95E1F7DF91CF91089580935F037093C2
:105210006103609360038091B007843001F582E000
:105220008093E9008FEF9091E800815095FD06C0D2
:1052300095ED9A95F1F700008111F5CF8091E80086
:1052400085FF0DC040E050E063E070E08FE593E043
:105250000E94B82A8091E8008E778093E800089534
:10526000BC0184E00C940529BC0183E00C94052961
:1052700008958091AF07811109C00E94492C0E94B6
:10528000A62C8091E20084608093E2000895109241
:10529000AF0708950C940A286091AC0781E0611172
:1052A00001C080E00C94F5270E9439289091B00746
:1052B00081E0943009F080E06091AC070C94FA270B
:1052C00042E061EC81E00E94C22B42E261EC82E0AC
:1052D0000E94C22B9091B00781E0943009F080E0E9
:1052E0006091AC070C9403288091B207833009F4D5
:1052F00061C030F4813071F0823009F49AC00895B1
:105300008A3009F486C08B3009F46CC0893009F00A
:10531000A8C020C08091B107813A09F0A2C0809155
:10532000E800877F8093E8008091B5079091B607E9
:10533000892B21F460E282E693E003C060E080E024
:1053400090E070E00E94032B8091E8008B778093BF
:10535000E80008958091B107813209F082C0809100
:10536000B5079091B607029708F07BC08091E800DE
:10537000877F8093E8008091E80082FD05C08091DE
:10538000B0078111F8CF6DC02091F3008091F20039
:1053900090E0922B029731F48091F100813011F06E
:1053A000863021F48091F100809382038091E8009F
:1053B0008B7753C08091B107813A09F052C0809138
:1053C000B5079091B607892B09F04BC08091E80092
:1053D000877F8093E8008091E80080FFFCCF809178
:1053E000910136C08091B1078132D9F58091B5071E
:1053F0009091B607892BA9F58091E800877F80936B
:10540000E8000E94F72B8091B307809391010C94E0
:10541000A00E8091B107813221F58091E800877F4D
:105420008093E8000E94F72B8091B4078093830358
:1054300008958091B107813AA1F48091E800877FB7
:105440008093E8008091E80080FFFCCF8091830387
:105450008093F1008091E8008E778093E8000C94AF
:10546000F72B089584B7877F84BF0FB6F894A8956B
:1054700080916000886180936000109260000FBE90
:1054800090E080E80FB6F8948093610090936100FB
:105490000FBE0C9405280E94492C0E94A62CE2EE17
:1054A000F0E080818460808378940C943B2F85E8C1
:1054B00091E00C94D626089508950C945F2A292F24
:1054C000332723303105C9F060F42130310581F0F4
:1054D0002230310509F044C08BE390E02BE73EE039
:1054E00043C021323105E1F02232310549F138C0A3
:1054F00082E190E026EB3EE037C0992781309105AC
:1055000049F028F0029761F5E9E5FEE005C0E7E71C
:10551000FEE002C0EBE6FEE0849190E09F0124C033
:105520006115710541F061307105D1F489E090E0B9
:1055300026EA3EE019C089E090E02DE83EE014C084
:105540006115710541F06130710551F48DE690E00F
:1055500028EC3EE009C080E490E025E33FE004C091
:1055600080E090E020E030E0FA013183208308956C
:10557000CF92DF92EF92FF920F931F93CF93DF931F
:10558000EC018B017A010E94162C811133C0E114C9
:10559000F10439F0F70180819181081B190BC80FC4
:1055A000D91FC12CD12C0115110519F18091E800EA
:1055B00085FD16C08091E8008E778093E800E114A5
:1055C000F10449F0F70180819181C80ED91ED18282
:1055D000C08285E00FC00E94162C882321F30AC0E8
:1055E00089918093F10001501109FFEFCF1ADF0A72
:1055F000DACF80E0DF91CF911F910F91FF90EF9074
:10560000DF90CF9008952091B7073091B807261703
:10561000370748F06115710539F42091E8002E77BD
:105620002093E80001C0B901FC0120E0611571057B
:1056300079F18091B0078823F1F18530F1F1809103
:10564000E80083FD3CC08091E80082FD2EC080917F
:10565000E80080FFEBCF2091F3008091F20090E012
:10566000922B6115710551F08830910538F4219124
:105670002093F100615071090196F3CF21E0089762
:1056800009F020E08091E8008E778093E800CECF8B
:105690002111CFCF0AC08091B007882361F08530F7
:1056A00061F08091E80083FD0AC08091E80082FFEC
:1056B000F2CF80E0089582E0089583E0089581E0CC
:1056C00008952091B7073091B8072617370748F09B
:1056D0006115710539F42091E8002E772093E800D8
:1056E00001C0B901FC0120E06115710591F18091C3
:1056F000B007882309F440C0853009F43FC0809189
:10570000E80083FD3DC08091E80082FD2FC08091BC
:10571000E80080FFE9CF2091F3008091F20090E053
:10572000922B6115710559F08830910540F4249150
:105730002093F1003196615071090196F2CF21E07A
:10574000089709F020E08091E8008E778093E800C8
:10575000CBCF2111CCCF0AC08091B007882361F054
:10576000853061F08091E80083FD0AC08091E800F7
:1057700082FFF2CF80E0089582E0089583E00895EB
:1057800081E00895982F973068F59093E900981775
:1057900039F07091EC002091ED005091F00003C0C1
:1057A000242F762F50E021FD02C09F5FECCF309177
:1057B000EB003E7F3093EB003091ED003D7F309366
:1057C000ED003091EB0031603093EB007093EC0012
:1057D0002093ED005093F0002091EE0027FDE5CFDF
:1057E00080E008958F708093E90081E008958091B2
:1057F000B10787FF11C08091E80082FD05C080914C
:10580000B0078111F8CF11C08091E8008B770BC0F1
:105810008091B007882349F08091E80080FFF8CF9D
:105820008091E8008E778093E80008952091E4004D
:105830003091E50095E64091EC00842F817040FFA7
:1058400023C08091E80080FD1DC08091B0078823AF
:1058500099F0853099F08091EB0085FD11C0409161
:10586000E4005091E5002417350729F3915011F019
:105870009A01E1CF84E0089582E0089583E00895DD
:1058800081E0089580E008954091E80042FFDDCF77
:1058900008950E94B72C0E94BF2CE0EEF0E08081BA
:1058A00081608083E8EDF0E080818F77808319BC90
:1058B000A7EDB0E08C918E7F8C9380818F7E80836A
:1058C0001092AF0708950F931F93CF93DF930E9419
:1058D000B72C0E94BF2CC8EDD0E088818F778883D9
:1058E00088818068888388818F7D888319BC109225
:1058F000B0071092AC071092AE071092AD0700EE01
:1059000010E0F80180818B7F8083888181608883AB
:1059100042E060E080E00E94C22BE1EEF0E0808196
:105920008E7F8083E2EEF0E08081816080838081E1
:1059300088608083F80180818E7F80838881806188
:105940008883DF91CF911F910F910895E8EDF0E0EA
:1059500080818F7E8083E7EDF0E0808181608083AD
:1059600084E082BF81E08093AF070C94632CE8ED64
:10597000F0E080818E7F80831092E2000895109283
:10598000DA001092E10008951F920F920FB60F9265
:1059900011242F933F934F935F936F937F938F9334
:1059A0009F93AF93BF93EF93FF938091E10082FFAA
:1059B0000BC08091E20082FF07C08091E1008B7FE5
:1059C0008093E1000E943A2F8091DA0080FF1FC08F
:1059D0008091D80080FF1BC08091DA008E7F809379
:1059E000DA008091D90080FF0DC080E189BD82E19D
:1059F00089BD09B400FEFDCF81E08093B0070E940D
:105A0000392905C019BC1092B0070E94472980911E
:105A1000E10080FF19C08091E20080FF15C08091F5
:105A2000E2008E7F8093E2008091E20080618093AB
:105A3000E2008091D80080628093D80019BC85E094
:105A40008093B0070E944C298091E10084FF30C010
:105A50008091E20084FF2CC080E189BD82E189BD94
:105A600009B400FEFDCF8091D8008F7D8093D800CF
:105A70008091E1008F7E8093E1008091E2008F7E33
:105A80008093E2008091E20081608093E200809147
:105A9000AC07882311F084E007C08091E30087FD04
:105AA00002C081E001C083E08093B0070E945429C6
:105AB0008091E10083FF29C08091E20083FF25C02F
:105AC0008091E100877F8093E10082E08093B007BE
:105AD0001092AC078091E1008E7F8093E10080916D
:105AE000E2008E7F8093E2008091E20080618093EB
:105AF000E20042E060E080E00E94C22B8091F00072
:105B000088608093F0000E944A29FF91EF91BF9135
:105B1000AF919F918F917F916F915F914F913F9145
:105B20002F910F900FBE0F901F9018951F920F92FC
:105B30000FB60F9211242F933F934F935F936F9360
:105B40007F938F939F93AF93BF93CF93DF93EF9305
:105B5000FF93C091E900CF708091EC00D82FD170F5
:105B600080FDD0E81092E9008091F000877F80935B
:105B7000F00078940E94DA2D1092E9008091F000F4
:105B800088608093F000CD2BCF70C093E900FF9127
:105B9000EF91DF91CF91BF91AF919F918F917F91C5
:105BA0006F915F914F913F912F910F900FBE0F908A
:105BB0001F9018951F93CF93DF93CDB7DEB7AA97A9
:105BC0000FB6F894DEBF0FBECDBFE1EBF7E08091DA
:105BD000F100819327E0E93BF207C9F70E9474299D
:105BE0008091E80083FF2EC18091B1079091B207A8
:105BF000492F50E04A30510508F024C1FA01EE590E
:105C0000FF4F0C94812F803821F0823809F01AC19F
:105C100008C08091AD079091AE07992389F082600A
:105C20000FC08091B5078F70873008F00BC180934B
:105C3000E9008091EB0085FB882780F91092E9004C
:105C40009091E800977F9093E8008093F100109284
:105C5000F100D1C0282F2D7F09F0F4C0882319F05E
:105C6000823061F0EFC08091B307813009F0EAC063
:105C7000933009F080E08093AE072EC08091B30787
:105C800081112AC08091B5078F702FEF280F263021
:105C900008F0D8C08093E9002091EB0020FF1CC0E1
:105CA000933021F48091EB00806214C09091EB005E
:105CB00090619093EB0021E030E0A90102C0440F15
:105CC000551F8A95E2F74093EA001092EA0080910E
:105CD000EB0088608093EB001092E9008091E8006F
:105CE000877F8093E8000E94F72BACC08111AAC087
:105CF0001091B3071F778091E3008078812B809308
:105D0000E3008091E800877F8093E8000E94F72BF2
:105D10008091E80080FFFCCF8091E3008068809351
:105D2000E300111102C082E001C083E08093B0075C
:105D300089C08058823008F085C08091B307909167
:105D4000B4078C3D53E0950779F583E08A838AE2B6
:105D500089834FB7F894DE01139620E03EE051E2CC
:105D6000E32FF0E050935700E49120FF03C0E29549
:105D7000EF703F5FEF708E2F90E0EA3010F0C79623
:105D800001C0C0968D939D932F5F243149F74FBF7B
:105D90008091E800877F8093E8006AE270E0CE019E
:105DA00001960E94032B16C06091B5077091B6074B
:105DB000AE014F5F5F4F0E945D2ABC01892B09F441
:105DC00041C09091E800977F9093E80089819A8183
:105DD0000E94612B8091E8008B778093E80032C0AD
:105DE000803881F58091E800877F8093E80080917A
:105DF000AC078093F1008091E8008E7772CF81111B
:105E000021C08091B3079091B40799270297D4F4E9
:105E10008091E800877F8093E8008091B3078093AA
:105E2000AC070E94F72B8091AC07811106C08091CE
:105E3000E30087FD02C081E001C084E08093B007E9
:105E40000E9460298091E80083FF0AC08091E800E9
:105E5000877F8093E8008091EB0080628093EB0065
:105E6000AA960FB6F894DEBF0FBECDBFDF91CF91DB
:105E70001F9108950895CF938091B0078823A1F0D2
:105E8000C091E900CF709091EC00892F817090FD56
:105E900080E8C82B1092E9008091E80083FD0E9401
:105EA000DA2DCF70C093E900CF9108950E94492C5C
:105EB0001092B00708958091E300881F8827881FFB
:105EC0000895991B79E004C0991F961708F0961B56
:105ED000881F7A95C9F780950895AA1BBB1B51E1CD
:105EE00007C0AA1FBB1FA617B70710F0A61BB70B4A
:105EF000881F991F5A95A9F780959095BC01CD01EF
:105F00000895EE0FFF1F0590F491E02D0994FB0119
:105F1000DC0102C005900D9241505040D8F7089521
:105F2000FB01DC0104C08D910190801921F44150E6
:105F30005040C8F7881B990B0895FB01DC0102C093
:105F400001900D9241505040D8F70895F999FECF35
:105F500092BD81BDF89A992780B50895A8E1B0E077
:105F600042E050E00C94DA2F262FF999FECF92BD33
:105F700081BDF89A019700B4021639F01FBA20BD0E
:105F80000FB6F894FA9AF99A0FBE08950396272F40
:105F90000E94B52F0E94B42F252F0E94B52F242FC9
:105FA0000C94B52F0196272F0E94B52F0C94B42F77
:105FB000DC01CB01FC01F999FECF06C0F2BDE1BDC9
:105FC000F89A319600B40D9241505040B8F70895B8
:045FD000F894FFCF73
:105FD4000000EC07000000000000000000000000CA
:105FE4000000000000000000FF07000000000000A7
:105FF4000000000000000000000000000000120883
:10600400000000000000000000000000000000008C
:1060140000000000DA07000000000000000000009B
:106024000000000000000000C800AE023632333128
:10603400F6F7F50100000001000000000000000573
:106044000100000004060000000000000021007FA1
:10605400220007FFFFC028C428382934293029C367
:106064002801F533F731F63236E200E900EA00B5EB
:1060740000B600B700CD008301CC008A01920194E0
:10608400012102230224022502260227022A02B346
:1060940000B4006F007000818283E200E900EA002E
:1060A400B500B600B700CD008301CC008A0192018F
:1060B40094012102230224022502260227022A0235
:1060C400B300B4006F0070008182836697C63435D4
:1060D400E80200081018202830383830282018101A
:0260E4000800B2
:00000001FF
